:100000003BC055C054C015C64DC5E6C58BC5B7C568
:100010001CC5C8C44CC09DC64AC0DFC683C047C00B
:1000200046C045C044C030313233343536373839B4
:1000300041424344454600000001000800400000E2
:1000400001000400000100080020004000800000C2
:100050000100041B5B25643B256448001B5B3F32A9
:10006000356C001B5B3F323568001B5B25646D00FF
:100070001B5B324A001B630011241FBECFE5D4E096
:10008000DEBFCDBF10E0A0E6B0E0EEE7F0E102C0D9
:1000900005900D92A036B107D9F711E0A0E6B0E0C7
:1000A00001C01D92A23DB107E1F759D0E7C7A8CF23
:1000B00033983798089596B1987F982B96B90895FC
:1000C00097B18295880F880F807C9F73982B97B982
:1000D000089597B18F71907E892B87B90895349ACE
:1000E000369A089586B19927807490700895109279
:1000F000B10197B18F71907E892B87B9349A369A66
:100100003699FECF24B185B19927982F88273327B8
:10011000822B932B0895EBDF96958795969587957F
:10012000992708951F920F920FB60F9211248F9363
:100130008FEF8093B1018F910F900FBE0F901F90A2
:100140001895379A359886B1887F866086B981E0A0
:10015000B7DF3D98339A1092B10178940895CAEFB1
:10016000D3E0DEBFCDBFB6D68FE896E0E6D08ED521
:10017000E8DF14BA15BA85E09EDF81E0A1DF92E0E6
:10018000C92ED12CCC0EDD1E86E6882E912C8C0E2D
:100190009D1E5E010894A11CB11CF6011192E81588
:1001A000F905E1F7198200E010E005C0F601EF0D56
:1001B000F11D89818083F02EC50145D60F5F1F4F49
:1001C0008823A1F700E010E004C0A9D58FE190E0FA
:1001D00000D3F601E00FF11D80810F5F1F4F8823D0
:1001E000A1F7DBCFFC018FB7F89471836083538351
:1001F000428317821682158214828FBF0895CF938F
:10020000DF93DC014FB7F894EC018C819D81892B41
:1002100011F4E0E01CC0FD0186819781ED91FC9115
:100220001197E80FF91FE0810196ED019F838E83FE
:100230002A813B818217930720F0821B930B9F83B7
:100240008E83ED018C819D8101979D838C834FBFAF
:100250008E2F9927DF91CF910895FC014FB7F89425
:100260008481958168177907B0F486819781860F1C
:10027000971F97838683228133818217930720F00B
:10028000821B930B9783868384819581861B970BB2
:100290009583848302C0158214824FBF0895FC01A8
:1002A000CB014FB7F8942681378162817381820F29
:1002B000931F93D60190F081E02DE80FF91F808104
:1002C0004FBF992708951F93CF93DF93EC01162F0B
:1002D0004FB7F8942C813D816A817B8126173707BF
:1002E00098F48E819F81820F931F77D6E881F981E0
:1002F000E80FF91F10838C819D8101969D838C836B
:100300004FBF8FEF90E003C04FBF80E090E0DF91E0
:10031000CF911F910895FC018FB7F8948FBF828110
:10032000938124813581821B930B0895FC018FB743
:10033000F894158214828FBF089590936100809382
:10034000600008951F93182F8A3031F4E091600007
:10035000F09161008DE00995E0916000F0916100FD
:10036000812F09951F910895CF93DF93EC01892B7D
:1003700019F405C02196E6DF88818823D9F7DF913B
:10038000CF910895EF92FF920F931F93CF93DF9336
:100390007A010097C1F0EC01680F791FC617D707E3
:1003A00019F089918823D1F700E010E009C0888115
:1003B000882311F0219601C080E2C4DF0F5F1F4F38
:1003C0000E151F05A1F7DF91CF911F910F91FF909F
:1003D000EF900895CF93DF93EC01892B11F406C0C1
:1003E000B1DFFE01219684918823D1F7DF91CF916F
:1003F00008958AE0A7DF0895E82FFF27EF70F070D7
:10040000EA5DFF4FE4918E2F9DDF08951F93182F13
:1004100082958F70F1DF812FEFDF1F9108950F9389
:100420001F938C01812F9927F1DF802FEFDF1F9120
:100430000F910895EF92FF920F931F937B018C0110
:10044000C801AA27BB27EBDFC701E9DF1F910F9186
:10045000FF90EF9008952F923F924F925F926F928C
:100460007F928F929F92AF92BF92CF92DF92EF9244
:10047000FF920F931F93CF93DF93CDB7DEB7A4976F
:100480000FB6F894DEBF0FBECDBF4BA32CA3270140
:100490003801442351F017FF08C0EE24FF248701E0
:1004A000E418F5080609170902C08301720169A35F
:1004B00090E02BA1211191E0E9A1E91BE150EAA311
:1004C00018A2882E992487FC9094A92CB92CC801D5
:1004D000B701A501940195D5FB01EF70F070EA5DBD
:1004E000FF4F64916F8FC801B701A501940189D5B1
:1004F00069017A012EE1222E312C2C0E3D1E20C0E6
:10050000C114D104E104F104A9F0C701B601A501A9
:10051000940177D5FB01EF70F070EA5DFF4F6491B5
:10052000F1016083C701B601A50194016AD5690193
:100530007A0103C02CA1F10120830894210831081D
:1005400081010F5F1F4F8AA181508AA38F3FC1F69F
:100550009BA19923B1F077FE03C081018DE20AC00F
:10056000411451046104710419F081018BE202C04D
:10057000810180E2F801808304C0F80181918F013C
:10058000E1DEF9A1F150F9A3FF3FB9F7A4960FB648
:10059000F894DEBF0FBECDBFDF91CF911F910F91B9
:1005A000FF90EF90DF90CF90BF90AF909F908F9093
:1005B0007F906F905F904F903F902F9008959F9203
:1005C000AF92BF92CF92DF92EF92FF920F931F9361
:1005D000CF93DF93CDB7DEB722970FB6F894DEBF87
:1005E0000FBECDBF9888C988DA88CE0143969A831A
:1005F000898304C0882309F465C0A4DE96012F5FB7
:100600003F4F992021F0F6016901849103C0F60162
:1006100080816901853271F72F5F3F4F992021F06A
:10062000F6016901849103C0F60180816901843675
:10063000A1F0883719F0833601F707C0E12C60E19B
:10064000F62E50E1A52EB12C0FC0E981FA81329629
:10065000FA83E98332978081D0CF40E1E42E47E2EC
:10066000F42E3AE0A32EB12CE981FA813296FA8376
:10067000E983129102918436A1F417FF0BC0109503
:1006800001951F4F8DE25EDE05C0C7016AE070E094
:10069000A4D47B01F2E0EF16F10418F00E151F054B
:1006A000A0F3C801B70199D4CB01A6DEC801B701F8
:1006B00094D48C01C701B50190D47B01672B09F458
:1006C0009DCFEFCF80E090E022960FB6F894DEBF8A
:1006D0000FBECDBFDF91CF911F910F91FF90EF9093
:1006E000DF90CF90BF90AF909F900895089583B70B
:1006F000887F826083BF12BE89B7816089BF1092F4
:10070000B2011092B3011092B4011092B501089594
:100710008EB5887F83608EBD1DBC1CBC89B784608C
:1007200089BF089585B5887F846085BD14BC89B76D
:10073000806489BF1092BA011092BB011092BC0173
:100740001092BD01089593B7987F982B93BF089599
:100750009EB5987F982B9EBD089595B5987F982B50
:1007600095BD0895E3B7FF27E770F070EE0FFF1F08
:10077000E95CFF4F859194910895EEB5FF27E770EE
:10078000F070EE0FFF1FE95CFF4F85919491089583
:10079000E5B5FF27E770F070EE0FFF1FED5BFF4F31
:1007A000859194910895873040F4E82FFF27EE0F4C
:1007B000FF1FEE59FF4F718360830895873040F427
:1007C000E82FFF27EE0FFF1FEE59FF4F1182108217
:1007D0000895EF92FF920F931F93CF93DF93EC0155
:1007E00012B71092B6011092B7011092B801109290
:1007F000B901B8DF9C014427552760E072E18AE720
:1008000090E021D4CA01B901693B2DE8720726E0C6
:10081000820720E0920770F427E2C131D20750F43A
:100820009E0144275527BAD328EE33E040E050E03C
:10083000E8D321C028EE33E040E050E0E2D3CA0123
:10084000B9019E0144275527A9D39B01AC0113C0D0
:100850008091B6019091B701A091B801B091B90112
:1008600085B78F7885BF85B7806885BF889585B740
:100870008F7785BF06C0210F311D411D511D7901A4
:100880008A012091B6013091B7014091B801509191
:10089000B90182B79927AA27BB27542F432F322F9C
:1008A0002227822B932BA42BB52B8E159F05A007F7
:1008B000B10770F2DF91CF911F910F91FF90EF90F0
:1008C00008951092B2011092B3011092B4011092E7
:1008D000B50108956091B2017091B3018091B401A6
:1008E0009091B50108951092BA011092BB01109237
:1008F000BC011092BD0108956091BA017091BB01D5
:100900008091BC019091BD010895893031F48FB57B
:1009100082608FBD8FB58E7F0AC08A3019F48FB583
:10092000826002C08FB58D7F8FBD8FB581608FBD16
:100930001BBC1ABC19BC18BC08952FB52E7F2FBD47
:100940002FB522602FBD2EB528602EBD2EB520619B
:100950002EBD97BD86BD1BBC1ABC19BC18BC089522
:100960008FB580688FBD8FB58F7B8FBD08958FB594
:1009700080628FBD8FB58F7E8FBD08958FB58F77C5
:100980008FBD8FB58F7B8FBD08958FB58F7D8FBD48
:100990008FB58F7E8FBD08959BBD8ABD089599BD8B
:1009A00088BD08951F920F920FB60F9211242F93B6
:1009B0003F934F935F936F937F938F939F93AF93E7
:1009C000BF93EF93FF938091B2019091B301A091F7
:1009D000B401B091B5010196A11DB11D8093B20182
:1009E0009093B301A093B401B093B5018091B60187
:1009F0009091B701A091B801B091B9010196A11DE4
:100A0000B11D8093B6019093B701A093B801B09344
:100A1000B9018091620090916300892B29F0E091E7
:100A20006200F09163000995FF91EF91BF91AF9142
:100A30009F918F917F916F915F914F913F912F91F6
:100A40000F900FBE0F901F9018951F920F920FB628
:100A50000F9211242F933F934F935F936F937F9344
:100A60008F939F93AF93BF93EF93FF938091640015
:100A700090916500892B29F0E0916400F091650068
:100A80000995FF91EF91BF91AF919F918F917F91C8
:100A90006F915F914F913F912F910F900FBE0F90EB
:100AA0001F9018951F920F920FB60F9211242F933B
:100AB0003F934F935F936F937F938F939F93AF93E6
:100AC000BF93EF93FF938091BA019091BB01A091E6
:100AD000BC01B091BD010196A11DB11D8093BA0169
:100AE0009093BB01A093BC01B093BD0180916C00B9
:100AF00090916D00892B29F0E0916C00F0916D00D0
:100B00000995FF91EF91BF91AF919F918F917F9147
:100B10006F915F914F913F912F910F900FBE0F906A
:100B20001F9018951F920F920FB60F9211242F93BA
:100B30003F934F935F936F937F938F939F93AF9365
:100B4000BF93EF93FF938091660090916700892B8C
:100B500029F0E0916600F09167000995FF91EF910F
:100B6000BF91AF919F918F917F916F915F914F91C5
:100B70003F912F910F900FBE0F901F9018951F92CD
:100B80000F920FB60F9211242F933F934F935F93C1
:100B90006F937F938F939F93AF93BF93EF93FF9345
:100BA0008091680090916900892B29F0E09168009C
:100BB000F09169000995FF91EF91BF91AF919F91DD
:100BC0008F917F916F915F914F913F912F910F90F6
:100BD0000FBE0F901F9018951F920F920FB60F9295
:100BE00011242F933F934F935F936F937F938F9332
:100BF0009F93AF93BF93EF93FF9380916A0090917F
:100C00006B00892B29F0E0916A00F0916B00099547
:100C1000FF91EF91BF91AF919F918F917F916F91D4
:100C20005F914F913F912F910F900FBE0F901F90AA
:100C300018951F920F920FB60F9211242F933F9386
:100C40004F935F936F937F938F939F93AF93BF93D4
:100C5000EF93FF9380916E0090916F00892B29F0A4
:100C6000E0916E00F0916F000995FF91EF91BF91B7
:100C7000AF919F918F917F916F915F914F913F9134
:100C80002F910F900FBE0F901F90189580E090E06D
:100C9000FC01EE0FFF1FEE59FF4F118210820196EB
:100CA00087309105A9F723DD33DD3CDD7894089585
:100CB0008FB58D7F8FBD8FB58E7F8FBD8FB58F77B1
:100CC0008FBD8FB58F7B8FBD8FB58F7D8FBD8FB55E
:100CD0008F7E8FBD08959093B0018093AF010895EA
:100CE000F3E0660F771F881F991FFA95D1F79B01D4
:100CF000AC01220F331F441F551F60507E4E8548A4
:100D00009F4F7FD12150304029B9232F332720BD59
:100D100008958FEB91E0089588EC91E00895982F65
:100D20008091BE018823E1F39CB91092BE01089521
:100D30001092C4011092C30108958091C301909153
:100D4000C401892B19F48FEF90E0089580E090E0C2
:100D500008951F920F920FB60F9211242F933F9375
:100D60004F935F936F937F938F939F93AF93BF93B3
:100D7000EF93FF936CB18091AF019091B001892BFB
:100D800039F0E091AF01F091B001862F09950EC0C6
:100D90008FEB91E098DA882349F48091D00190910B
:100DA000D10101969093D1018093D001FF91EF91F1
:100DB000BF91AF919F918F917F916F915F914F9173
:100DC0003F912F910F900FBE0F901F901895682F95
:100DD00088EC91E078DA992708951F920F920FB668
:100DE0000F9211242F933F934F935F936F937F93B1
:100DF0008F939F93AF93BF93EF93FF938091C7011E
:100E0000882369F08091CC019091CD01892B29F044
:100E100088EC91E0F4D98CB905C01092C7018FEF2E
:100E20008093BE01FF91EF91BF91AF919F918F9100
:100E30007F916F915F914F913F912F910F900FBED6
:100E40000F901F901895CF93DF93EC018091C10113
:100E50009091C201892B69F08091C3019091C401E6
:100E6000892B39F08FEB91E0CAD988838FEF90E01E
:100E700002C080E090E0DF91CF910895CF93DF939F
:100E8000CDB7DEB721970FB6F894DEBF0FBECDBF4A
:100E9000CE010196D8DF882319F48FEF9FEF02C0AF
:100EA0008981992721960FB6F894DEBF0FBECDBF7A
:100EB000DF91CF9108954FEF50E060E770E08FEB46
:100EC00091E090D940E450E06FE671E088EC91E069
:100ED00089D90895F0DF1092B0011092AF0188ED2A
:100EE0008AB960E875E280E090E0FADE8FEF8093E7
:100EF000BE011092C7011092D1011092D0017894D6
:100F000008958FEF8093C70188EC91E078D9982FEE
:100F10008091BE018823E1F39CB91092BE0108952F
:100F200077277F936F9399279F938F9383E590E023
:100F30009F938F9381E08F9342DB8DB79EB7079687
:100F40000FB6F8949EBF0FBE8DBF0895882319F089
:100F500083E690E002C08CE590E09F938F9381E060
:100F60008F932DDB0F900F900F90089599279F93EB
:100F70008F938AE690E09F938F9381E08F931FDB9E
:100F80000F900F900F900F900F90089580E790E0D2
:100F900021DA089585E790E01DDA0895629FD00177
:100FA000739FF001829FE00DF11D649FE00DF11D24
:100FB000929FF00D839FF00D749FF00D659FF00DD3
:100FC0009927729FB00DE11DF91F639FB00DE11DC0
:100FD000F91FBD01CF0111240895AA1BBB1B51E1CC
:100FE00007C0AA1FBB1FA617B70710F0A61BB70B99
:100FF000881F991F5A95A9F780959095BC01CD013E
:101000000895A1E21A2EAA1BBB1BFD010DC0AA1F49
:10101000BB1FEE1FFF1FA217B307E407F50720F061
:10102000A21BB30BE40BF50B661F771F881F991FDC
:101030001A9469F760957095809590959B01AC0125
:10104000BD01CF01089597FB092E05260ED057FD4F
:1010500004D0D7DF0AD0001C38F450954095309565
:1010600021953F4F4F4F5F4F0895F6F7909580952C
:0E107000709561957F4F8F4F9F4F0895FFCF72
:00000001FF
